:100000000C947603189518951895189518951895C9
:1000100018951895189518950C94B201189518957F
:10002000189518950C948F01189518951895189592
:100030000C944C0118951895189518950C9423015B
:100040001895189518951895189518951895189548
:100050001895189518951895189518951895189538
:100060001895189518951895189518951895189528
:10007000DC9A03E00A95F1F70000DC9808951BB3C1
:10008000107F02950F70102B1BBBF2CF8A93802F2D
:10009000112311F0DD9A01C0DD981BD08295807F7D
:1000A000082F17D00AEF00000A95E9F78991089503
:1000B00010E0ECCF11E0FDCFBA93AA93D80101C0B4
:1000C000BBD00D910023E1F7A991B991089501D01A
:1000D00001C0D5CF03ED10E301501040E9F700C097
:1000E00000000895F7DF16D015D014D000E2EFDF3E
:1000F00008E20FD00CE00DD001E00BD0EBDF00E800
:1001000008D00CE811E0D8DF00EC03D000E911E0E2
:10011000D3CFCECF00E3DBCF0E9498032897DAD26B
:100120005888498890E083E0ACEBB1E077D038F5AF
:10013000552081F000E010E020E030E040E050E0A9
:1001400060EF7FE3BFD2C6D285E004C0A4ECB1E08B
:10015000C0D2839565D0ACECB1E00E94D506B0F377
:100160005FD0A4ECB1E05AD028F4ACEBB1E0B1D24E
:100170008A95F6CF55D050D050F45FD0FBCF9883FE
:1001800099839A839B839C839D839E839F8307E0AF
:10019000401671F445D0A4EEB1E00E9402059AD257
:1001A0003BD030F440D049D0933014F08A9590E0A1
:1001B000662419C035D00E947304A02F005D3CD086
:1001C000691611F40EE238D00A2F1A2F110F110BF5
:1001D000212F312F0E946004DE010E949605A4EDBC
:1001E000B1E077D26394762C770C770855246414A9
:1001F000750404F320D0982F990F990B880F991F3D
:10020000880F991F04E911E0080F191F55DF13D05B
:100210002896EAE00C94A103A4EDB1E00C94FB064F
:1002200002D07F810895088119812A813B814C8108
:100230005D816E81089500E23DCFACEDB1E040D22A
:1002400049D293950895AED002A913A981D002ABEB
:1002500013AB789400A911A97BD000AB11AB06AD0C
:10026000039506AF093120F000E006AF01E006ABD0
:1002700007A9002329F007A90A9507AB959A01C0A1
:10028000959800AD002329F000AD0A9500AF969A2D
:1002900001C0969860D01895FA93EA934A933A93DE
:1002A0002A931A930A934FB7ECEFF1E004A115A13A
:1002B00026A137A12CD005A90130C1F404A1048BDB
:1002C000158B268B378B04B515B500A711A702A98E
:1002D00013A902A713A708B707FF06C000A511A519
:1002E0000030104808F458D002E005AB08B703FF0F
:1002F00005C004A115A10BD008E008BF4FBF0991AC
:100300001991299139914991E991F991189520D044
:100310002F4F3F4F04A315A326A337A3089546D01C
:10032000EBE3F2E00081118113D000831183789414
:1003300000913502039500933502009135020A3F82
:1003400030F000E00093350201E000933602A2CFC6
:100350000F5F1F4F08952FBF099119912991E991BE
:10036000F99108951FD0009180001091810004A799
:1003700015A700913B0210913C0206A717A7009118
:100380007C0002FF05C000A511A5103808F404D0B8
:1003900001E0FD9600837ECF02A513A5D9DF02A759
:1003A00013A7089503D0ECEFF1E00895FA93EA93D0
:1003B0002A931A930A932FB708951B2F2A2F40E0F0
:1003C00000E054E0459FF001E35CFD4F5DD14395B3
:1003D0004430B0F3ECEFF1E0DF01DC960C9303AFB7
:1003E00000A301A302A303A300AFA22FB12F08957E
:1003F0000E949C038CEF91E000913602002321F0D3
:1004000000E000933602D9DF00913902002309F49D
:1004100075C000E00093390200933502ADE3B2E00D
:10042000FC0166A577A504A515A50D931D936D93F5
:100430007C9313970D911D912D913C911397FD0184
:100440003AD11DD1408151816281738127D1A801A8
:10045000B901415C5D41644F70404F375C40604082
:10046000704008F04BC04091380254E0459FE00DC9
:10047000F11D4085518562857385FC0100A011A0A6
:1004800022A033A0041A150A260A370A00A211A2D4
:1004900022A233A240A151A162A173A1400F511F1A
:1004A000621F731F40A351A362A373A344AD542FD3
:1004B000539554AF54E0459FA00DB11DFD0121D0CF
:1004C00000913802043018F000E000933802FC017B
:1004D00003AD039503AF03AD043070F053AF00A13B
:1004E00011A122A133A1C9D0ACEEB1E0E9D0FC0149
:1004F00008D0BED00AEF01C003E500AFE4E00C94E1
:10050000A50300871187228733870895289701E084
:1005100007B908E002BB0FE30ABB00EE01BB07E02E
:1005200003BFE0DD8CEF91E000E040E854E86EE6C8
:1005300071E4FC01A9D09CD0469A04AB01E005AB64
:100540000EBD08E809BF01E000938A0004E20093B1
:100550007D0078941AC049E147AB8FD0BBD08201AF
:1005600093018BD0DC011896ABD0ACD092D0429BDB
:1005700004C0A4EFB1E0A4D08CD004E8A6D000E081
:1005800092D004ECA2D001E08ED032DF0091320292
:100590000023F1F000E00093320202B718B711FF18
:1005A00003C002E008BF0FEF10E012BF429B07C07C
:1005B000043170F4979808B1087F08B904C0093273
:1005C00038F0979A429A01E000933102109330027A
:1005D00009B70F7709BF00913102002359F4FC01DC
:1005E00000A911A9043620E0104020F001E005AB7D
:1005F00020AB21AB09B7006809BF0091310202307E
:1006000021F6FC0162A573A500A511A5048F158F25
:10061000668F778F048D158D268D378D408D518D8A
:10062000628D738D2CD0448D558D668D778D408F66
:10063000518F628F738F4488558866887788408988
:10064000518962897389441A550A660A770A44896E
:10065000558966897789408B518B628B738B40E01B
:1006600045AB44A9442309F076CF01E004AB8DCF1C
:10067000448755876687778708950C947104041B17
:10068000150B260B370B0895008701870287038718
:100690000895FC01008311832283338344835583AF
:1006A0006683778308950A93FC010081118122817A
:1006B000338101D031CD44815581668177810895A0
:1006C0000C94BF05DE010C943706F2DC07E00A93B8
:1006D0000895F6DF088319832A833B834C835D8367
:1006E0006E837F83089500008895FECF0BE80DBFD1
:1006F00001E00EBFC0E5D1E00E940507002311F024
:100700000E9415070E9486020E9473030C947303D3
:100710004A952AF03695279517950795F9CF0895AC
:1007200030952095109501951F4F2F4F3F4F0895FD
:100730007A926A925A924A92BA93AA939A938A9315
:1007400008957F806E805D804C80BB81AA819981F5
:100750008881F0E0EC0FFD1FEF01089527973A9391
:100760002A931A930A934A930D903D91FD91ED912E
:100770000D911D912D911C9017973324222443E055
:10078000110C37941694000C331FFF1FEE1F001F2F
:10079000111F221F111C221C4A95A9F7220F111CA0
:1007A000221C14162406089411F488941394279597
:1007B0002B871A870987E887FF833E830D8249913B
:1007C00009911991299139910024EE27F3E0770FCF
:1007D00007947695000F111F221F331F441F551FCA
:1007E000661F771FEE1FFA95A9F7660F771FEE1F9A
:1007F0007F17EF07089411F4889471E067950895C6
:1008000067FD1AC0000F111F221F331F441F551F01
:10081000661F7150E040FF277130EF0769F084F7E1
:10082000669557954795379527951795079508F439
:1008300068947F5FEF4FF0CFF7E0F023F43021F4BE
:100840002EF003FD03C00BC008F409C0085F1F4F62
:100850002F4F3F4F4F4F5F4F6F4F7F4FEF4FFF2750
:100860007230EF0718F467FF772709C0F7E07F3F82
:10087000EF0728F06627552744279A018A01F3E0FD
:10088000660FE69577956795E69577956795579501
:1008900047953795279517950795FA95A9F7700D00
:1008A00008957FE7702960EF552744279A018A0150
:1008B0000895702D70786627F7CF7FEF6FEF08955A
:1008C000002437FB07F816F40E949003412F522FA3
:1008D000632F302F002711272227E4E07EE1E894E0
:1008E0009ACF0024F3CF70DF7F5FE34080F01124C4
:1008F0007F31E10570F007FC05C03FE72FEF1FEFE8
:100900000FEF089530E82227112700270895332795
:10091000FACF252F142F032F362F472F4F514195F4
:100920000E94880307FE08950C949003072EE62F7B
:10093000EE0F001CFFEFE03E0F0650F4E029E52B20
:10094000E42BE32BE22BE12BE02B8894B894089561
:10095000E05EE52BE42BE32BE22BE12BE02B19F0FF
:100960000894B894089588949894389408951796A4
:100970000C90EE91EE0F001CFFEFE03E0F0680F4AE
:10098000E0293E902E901E90E329E229E1293E9035
:100990002E901E90E329E229E1298894B8940895C5
:1009A000E05E3E902E901E90E329E229E1293E90E0
:1009B0002E901E90E329E229E129A9F2D1CF7FEF01
:1009C0006FEF0895D4DF13F0D0F308951796FC91DC
:1009D0001797F727A2F30895CADF51F00D911D91E3
:1009E0002D913D914D915D916D917C911797089559
:1009F0001796EC9117977E23089517967C91179779
:100A000052CF089593DFD8F2EBF231F3B0DFB8F2B2
:100A1000A3F3B9F32397E894A1DE17162E0638F551
:100A20000F82E88779877119E209EE23E1F49F9339
:100A3000BF933F92972F7991E991F991099019907D
:100A4000299039903694279417940794F795E79551
:100A5000779508F468949A95A9F79F91B8819B2798
:100A6000BF919F911EC0710DE21D2A9608CF1716E7
:100A70002E0661F0669557954795379527951795FA
:100A8000079508F468947F5FEF4FF1CF30240F8211
:100A9000E88779877991E991F991099019902990DE
:100AA0003990AAF0070F1E1F2F1F301D411D521D28
:100AB000631D0990E9917991C0F567955795479520
:100AC00037952795179507957F5FEF4FA4CE0717AA
:100AD0001E072F073005410552056305B9F0C8F41C
:100AE0000EF08894700BE10BF20B030A140A250A2E
:100AF000360A072F1E2F2F2F302D412D522D632DFB
:100B00000990E9917991F0E80F2685CE7727239611
:100B1000D2CE0EF40894070B1E0B2F0B300941099F
:100B2000520963090990E991799175CEF0E87F2720
:100B300069CF1DDF38F031F01796FC911797F078E8
:100B40007F2708953CCF13DFE8F3E3F31796FC917A
:100B50001797F0787F2708951796FC9117977F27AE
:100B600070787158A0CE1796FC9117977F277078F0
:100B7000A2CE2A96702DF5CF2A96702D9CCED6DE69
:100B800008F3BBF201F3F3DEE8F233F361F32397EA
:100B9000E894E4DD0324710DE21D7F5FE340FFEF85
:100BA0007D3CEF074CF3F7E07F3FEF0714F70F8230
:100BB000E8877987AF93BF939F938F934F92F7E026
:100BC000222411240024C001D001E8E03324772737
:100BD000499040FE08C0800FA11FB21F931F041E42
:100BE000151E261E371E000F111F221F331F441F04
:100BF000551F661F771F4694EA9559F7882309F019
:100C00006894FA9579F08A2FAB2FB92F902D012C8B
:100C1000122C232C012F122F232F342F452F562F28
:100C2000672FD3CF632D522D412D302D292F8D01CC
:100C30000990E991799167FF03C07F5FEF4F07C08B
:100C4000000F111F221F331F441F551F661F4F9097
:100C50008F919F91BF91AF91DECD89DE10F00BF0A7
:100C60006BCFADCE84DEE9F3E0F37DCF75CF5EDEF2
:100C7000C0F39BF3B9F37BDEA0F3BBF3B9F3239787
:100C8000E8946CDD032467FD0AC0000F111F221FCA
:100C9000331F441F551F661F7150E040F4CF3E8044
:100CA00037FC19C0F881FF0FF883F981FF1FF98322
:100CB000FA81FF1FFA83FB81FF1FFB83FC81FF1F6B
:100CC000FC83FD81FF1FFD83331C3E82F1E01F1A70
:100CD000F0E02F0AE4CF7150EC4F7119E2092AF4C9
:100CE000FFEF7D3CEF0708F447CFF7E07F3FEF07CA
:100CF0000CF03FCF0F82E88779879F93BF93AF9324
:100D00007991E991F9910990199029903990669516
:100D100057954795379527951795079536942794B6
:100D200017940794F795E7957795A7E09927B8E08A
:100D3000990F07171E072F07300541055205630558
:100D400040F0071B1E0B2F0B3009410952096309A4
:100D50009395000F111F221F331F441F551F661F3D
:100D6000BA9531F79A93AA9509F70A171A072A072D
:100D70003A074A075A076A0709F06894AF91BF918A
:100D80009F910991199129913991499159916991AD
:100D90000990E99179913FCDEADD59F11796FC91DF
:100DA0001797FF2332F108940895E1DD10F1BEDDBD
:100DB00000F191F3E72F1796FC91EF271AF417979C
:100DC000F71708953E902E901E90149741155205E6
:100DD00063057F0758F051F414963E902E901E90B4
:100DE0000E90001511052205330571F0772362F48A
:100DF00050F488940895BBDDE0F398DDD0F3D9DF9B
:100E0000C0F3089408950894089501E0089520E03F
:100E100006D0E9F70895259102D0E9F708952D93BA
:100E200001501040202F212B08958EE59EE0FC01FB
:100E300005911491FC013296A591B491FC01349670
:100E400025913491422F432B19F0F901E4DF01C0C1
:100E5000DEDF06961EE08A36910748F3089570009B
:100E60008C016A0E5900FC010000462E3A00502EFB
:100E70003A0047487A004D487A006B487A00487A31
:100E800020006D487A0073656B006D7320007573E8
:100E900020006E73200070732000FCA9F1D24D6217
:100EA000503F0000000000408F40000000000000A4
:100EB000F03F00000000000024409A999999999908
:100EC000B93F8DEDB5A0F7C6A03E000000000000C0
:0A0ED000D03F000000000000704059
:00000001FF
:00000001FF
